:020000040000FA
:100000000A128A11D32FFF1B0D2883137F18831721
:100010000008840A0319FF0A080000308A00040857
:10002000840A820700345234543443342F344C341D
:10003000433444342034773469347434683420349D
:1000400050344934433400346434643464342C34DC
:100050002034443444342F344D344D342F34593407
:100060005934203420340034203443346934723419
:1000700063347534693474342034443469346734F7
:100080006534733474340034483448343A346D344D
:100090006D343A347334733420342D345034503446
:1000A0002E345034003457346534643400345434BE
:1000B00075346534003446347234693400344D3458
:1000C0006F346E340034533475346E34003453342A
:0E00D0006134743400345434683475340034B0
:1000E00014340034073400340F307605F800003043
:1000F0007705F900760E0F39F000770EF039F0042D
:10010000770E0F39F100F030F11D0030F1040A30A4
:10011000F2000030F3000A128A15522578087007A1
:10012000F60079080318790A7107F7000800C92852
:10013000513083160313CA008030CB0008004D30C5
:1001400083160313CA008030CB00080045308316A5
:100150000313CA008030CB0008004130831603131C
:10016000CA008030CB000800593083160313CA0040
:100170008030CB000800493083160313CA0080305A
:10018000CB000800553083160313CA008030CB0023
:1001900008007108003A0319CE28E5287008013AD2
:1001A00003199828033A03199F28013A0319A6282E
:1001B000073A0319AD28013A0319B428033A031981
:1001C000BB28013A0319C228E52808008316031347
:1001D0008715071628308312031394008316031320
:1001E0009101831203135A08DE005B08DF005C08EC
:1001F000E0005D08E10002300310DE0DDF0DE00DD0
:10020000E10DFF3E031DFC286108F3006008F200C9
:100210005F08F1005E08F0000030F7000030F600E3
:100220000030F5006430F4000A128A15A8260A127C
:100230008A11730883120313D0007208CF0071086B
:10024000CE007008CD000130D4003130D3002D3005
:10025000D2000030D1000A128A11EC21831203135C
:100260004D08FF3E83160313930094010800F60126
:10027000F11F4129F009F109F00A0319F10AF60109
:10028000F60AF31F4C29F209F309F20A0319F30ADB
:100290000130F4007408F606F701F80170087104E3
:1002A00003198329F501F50AF11B622901300310B6
:1002B000F00DF10DFF3E031D57290130F4007408C5
:1002C000F507542901300310F70DF80DFF3E031D0B
:1002D000632971087302031D6F2970087202031CE1
:1002E00078297008F2027108031CF303F3027714F3
:1002F00001300310F10CF00CFF3E031D7929013091
:10030000F502031D6229760803198B29F709F809FC
:10031000F70A0319F80A7808F1007708F0000800D6
:1003200000300A128A151E250A128A118230F50041
:10033000DD30F400F40B9A29F50B9A299F2903303C
:100340000A128A1538250A128A112130F5007630F2
:10035000F400F40BA929F50BA929000003300A12B7
:100360008A1538250A128A114830F5006C30F400DD
:10037000F40BB829F50BB829000003300A128A15CE
:1003800038250A128A1102300A128A1538250A12F3
:100390008A1102300A128A1538250A128A11083089
:1003A0000A128A1538250A128A1100300A128A1593
:1003B00038250A128A110C300A128A1538250A12B9
:1003C0008A1100300A128A1538250A128A1106305D
:1003D0000A128A1538250800003083120313D8004A
:1003E0000030D7000030D6000030D50050084F0450
:1003F0004E044D040319432AD901D90AD01B0E2AF1
:100400000130FD000310CD0DCE0DCF0DD00DFD0B35
:10041000022A0130FD007D08D907FE290130FD00C8
:100420000310D50DD60DD70DD80DFD0B102A500891
:100430005402031D252A4F085302031D252A4E0886
:100440005202031D252A4D085102031C362A4D086D
:10045000D1024E08031C4E0FD2024F08031C4F0F4F
:10046000D3025008031C500FD4025514013003105E
:10047000D00CCF0CCE0CCD0CFF3E031D372A013023
:10048000D902031D0E2A5808D0005708CF0056087D
:10049000CE005508CD000800831603138701831290
:1004A0000313870183160313880183120313880142
:1004B0000030DD000130DC008630DB00A030DA00E7
:1004C0000A128A11E6200A128A110A128A11902150
:1004D0000A128A110A128A15FE250A128A110A12B4
:1004E0008A15E7260A128A110A128A1139230A127A
:1004F0008A110A128A111C240A128A110A128A15F8
:1005000008250A128A110A128A111A260A128A1159
:100510000A128A11B8220A128A110730F00000303C
:10052000F1000A128A1197200A128A11831203130A
:100530006D08831603134906031DA42A83120313AF
:100540006C088316031348060319742A0A128A11C9
:1005500013250A128A11831203136D0883160313DD
:10056000C900831203136C0883160313C800742A8E
:1005700083120313A11FD12AFF30F000FF30F100D6
:100580002108F3002008F2000A128A1552250A12E7
:100590008A11710883120313A1007008A0002D3086
:1005A000D22A2B30F9007908EE0006300310A30C94
:1005B000A20CFF3E031DD62A1930F0000030F100D6
:1005C0002308F3002208F2000A128A1552250A12A3
:1005D0008A11710883120313A3007008A200220875
:1005E0002304031DF72A3030F9007908C0001930C0
:1005F00022062304031D002B3230F9007908C000C5
:10060000323022062304031D092B3530F900790806
:10061000C0004B3022062304031D122B3730F90093
:100620007908C0000A30F0000030F1002108F30022
:100630002008F2000A128A15B5270A128A117008DA
:10064000303EF900790883120313BF000A30F0002E
:100650000030F1002108F3002008F2000A128A118C
:1006600037217008303EF900790883120313BE0069
:1006700008000A128A15B8240A128A11D030F00034
:100680000030F1000A128A15C6240A128A110030BD
:10069000F000F1000A128A15C6240A128A110A1201
:1006A0008A15B1240A128A11D130F0000030F1000D
:1006B0000A128A15C6240A128A110130F00000308D
:1006C000F1000A128A1573250A128A117108F700BF
:1006D0007008F6000A128A1174200A128A1177082B
:1006E00083120313ED007608EC000130F0000030B7
:1006F000F1000A128A1573250A128A117108F7008F
:100700007008F6000A128A1174200A128A117708FA
:1007100083120313EB007608EA000130F00000308A
:10072000F1000A128A1573250A128A117108F7005E
:100730007008F6000A128A1174200A128A117708CA
:1007400083120313E9007608E8000130F00000305E
:10075000F1000A128A1573250A128A11700883168D
:100760000313CA007108CB000130F0000030F10023
:100770000A128A1573250A128A117108F700700887
:10078000F6000A128A1174200A128A11770883125D
:100790000313E7007608E6000130F0000030F100B6
:1007A0000A128A1573250A128A117108F700700857
:1007B000F6000A128A1174200A128A11770883122D
:1007C0000313E5007608E4000130F0000030F1008A
:1007D0000A128A1573250A128A117108F700700827
:1007E000F6000A128A1174200A128A1177088312FD
:1007F0000313E3007608E2000A128A15BF240A12E6
:100800008A110A128A15B8240A128A11D130F0000E
:100810000030F1000A128A15C6240A128A1101302A
:10082000F0000030F1000A128A1573250A128A11AD
:100830000A128A15BF2408000A128A15B8240A125F
:100840008A11D030F0000030F1000A128A15C62457
:100850000A128A110730F0000030F1000A128A15DE
:10086000C6240A128A110A128A15B1240A128A11A0
:10087000D130F0000030F1000A128A15C6240A12A5
:100880008A110130F0000030F1000A128A15732538
:100890000A128A117108F7007008F6000A128A110C
:1008A00074200A128A11770883120313B3007608A2
:1008B000B2000130F0000030F1000A128A157325F1
:1008C0000A128A117108F7007008F6000A128A11DC
:1008D00074200A128A11770883120313B100760874
:1008E000B0000130F0000030F1000A128A157325C3
:1008F0000A128A117108F7007008F6000A128A11AC
:1009000074200A128A11770883120313AF00760845
:10091000AE000130F0000030F1000A128A15732594
:100920000A128A110130F0000030F1000A128A1513
:1009300073250A128A117108F7007008F6000A126E
:100940008A1174200A128A11770883120313AD00EA
:100950007608AC000130F0000030F1000A128A1570
:1009600073250A128A117108F7007008F6000A123E
:100970008A1174200A128A11770883120313AB00BC
:100980007608AA000130F0000030F1000A128A1542
:1009900073250A128A110130F0000030F1000A12AA
:1009A0008A1573250A128A11710883120313A50090
:1009B0007008A4000130F0000030F1000A128A151E
:1009C00073250A128A11710883160313CD0070086B
:1009D000CC000130F0000030F1000A128A157325B6
:1009E0000A128A110130F0000030F1000A128A1553
:1009F00073250A128A11710883120313A10070086B
:100A0000A0000030F000F1000A128A1573250A12C6
:100A10008A11710883120313A3007008A2000A123E
:100A20008A15BF240800F401F40A01300A128A155D
:100A30006B270A128A118312031347080A128A15B8
:100A400033260A128A118312031348080A128A15E0
:100A500033260A128A110430FB007B08F4000130AF
:100A60000A128A156B270A128A1183120313490886
:100A70000A128A1533260A128A11831203134A08AE
:100A80000A128A1533260A128A110730FB007B08E6
:100A9000F40001300A128A156B270A128A11831298
:100AA00003134B080A128A1533260A128A1183127D
:100AB00003134C080A128A1533260A128A110630CB
:100AC000FB007B08F40002300A128A156B270A1219
:100AD0008A118312031345080A128A1533260A1253
:100AE0008A118312031346080A128A1533260A1242
:100AF0008A110930FB007B08F40002300A128A15C3
:100B00006B270A128A118312031343080A128A15EB
:100B100033260A128A118312031344080A128A1513
:100B200033260A128A110C30FB007B08F4000230D5
:100B30000A128A156B270A128A11831203134108BD
:100B40000A128A1533260A128A11831203134208E5
:100B50000A128A1533260A128A11F401F40A0230A5
:100B60000A128A156B270A128A11831603134A0880
:100B7000F5004B08F6000A128A159F250A128A1101
:100B80000A30FB007B08F40001300A128A156B273B
:100B90000A128A11831203136E080A128A15332669
:100BA0000A128A11831203133E080A128A15332689
:100BB0000A128A11831203133F080A128A15332678
:100BC0000A128A110E30FB007B08F40001300A1271
:100BD0008A156B270A128A118312031340080A121E
:100BE0008A1533260A128A11831203136A086B04CA
:100BF000031D072E6C086D04031D072E0230F00044
:100C00000030F1000A128A1528270A128A111E30B4
:100C1000831203136A066B04031D08006C086D043D
:100C2000031D08000130F0000030F1000A128A159F
:100C3000282708000A30F0000030F1008312031367
:100C40006D08F3006C08F2000A128A15CC250A120E
:100C50008A117008303EF800780883120313CC0024
:100C60000A30F0000030F1006D08F3006C08F2006B
:100C70000A128A156C260A128A117008303EF80092
:100C8000780883120313CB000A30F0000030F10023
:100C90006B08F3006A08F2000A128A15CC250A12C2
:100CA0008A117008303EF800780883120313CA00D6
:100CB0000A30F0000030F1006B08F3006A08F2001F
:100CC0000A128A156C260A128A117008303EF80042
:100CD000780883120313C9000A30F0000030F100D5
:100CE0006908F3006808F2000A128A15CC250A1276
:100CF0008A117008303EF800780883120313C80088
:100D00000A30F0000030F1006908F3006808F200D2
:100D10000A128A156C260A128A117008303EF800F1
:100D2000780883120313C7000A30F0000030F10086
:100D30006708F3006608F2000A128A15CC250A1229
:100D40008A117008303EF800780883120313C60039
:100D50000A30F0000030F1006708F3006608F20086
:100D60000A128A156C260A128A117008303EF800A1
:100D7000780883120313C5000A30F0000030F10038
:100D80006508F3006408F2000A128A15CC250A12DD
:100D90008A117008303EF800780883120313C400EB
:100DA0000A30F0000030F1006508F3006408F2003A
:100DB0000A128A156C260A128A117008303EF80051
:100DC000780883120313C3000A30F0000030F100EA
:100DD0006308F3006208F2000A128A15CC250A1291
:100DE0008A117008303EF800780883120313C2009D
:100DF0000A30F0000030F1006308F3006208F200EE
:100E00000A128A156C260A128A117008303EF80000
:100E1000780883120313C1000A30F0000030F1009B
:100E20003308F3003208F2000A128A15CC250A12A0
:100E30008A117008303EF800780883120313BD0051
:100E40000A30F0000030F1003308F3003208F200FD
:100E50000A128A156C260A128A117008303EF800B0
:100E6000780883120313BC000A30F0000030F10050
:100E70003108F3003008F2000A128A15CC250A1254
:100E80008A117008303EF800780883120313BB0003
:100E90000A30F0000030F1003108F3003008F200B1
:100EA0000A128A156C260A128A117008303EF80060
:100EB000780883120313BA000A30F0000030F10002
:100EC0002F08F3002E08F2000A128A15CC250A1208
:100ED0008A117008303EF800780883120313B900B5
:100EE0000A30F0000030F1002F08F3002E08F20065
:100EF0000A128A156C260A128A117008303EF80010
:100F0000780883120313B8000A30F0000030F100B3
:100F10002D08F3002C08F2000A128A15CC250A12BB
:100F20008A117008303EF800780883120313B70066
:100F30000A30F0000030F1002D08F3002C08F20018
:100F40000A128A156C260A128A117008303EF800BF
:100F5000780883120313B6000A30F0000030F10065
:100F60002B08F3002A08F2000A128A15CC250A126F
:100F70008A117008303EF800780883120313B50018
:100F80000A30F0000030F1002B08F3002A08F200CC
:100F90000A128A156C267008303EF8007808831211
:100FA0000313B40008008313D230FD000030FE00AC
:100FB0007030FF00CE3084000A128A15FB240A121A
:100FC0008A116F30FD000C30FE00EA30FF00623005
:100FD00084000A128A15FB240A128A11A0308400A8
:100FE000CE300A128A15CE240A128A1120308400CB
:100FF0004D300A128A15CE2483010A128A114C2A16
:101962000A128A15D62483160313911408000A1248
:101972008A15D62483160313111408000A128A1535
:10198200D62483160313111508000A128A15D624C9
:101992007008831203139300080064008001840A14
:1019A2000406031900340406CF2C8316031311080E
:1019B2001F39031DD62C141D0800D62C00300A1224
:1019C2008A1538250A128A1501300A128A15382515
:1019D200080013340034073400341B340034153447
:1019E20000342A3400341E34003420347E088A0045
:1019F2007F088200F7240A128A158000840A0408EC
:101A02007D0603190034FF0A0319FE0AFB2C01307C
:101A1200831203132405A80000302505A900250818
:101A2200F1002408F0000310F10CF00C01307005F5
:101A3200A60000307105A7000800F000701C252DDB
:101A4200831203130816282D831203130812F01CA5
:101A52002C2D88162D2D8812701D312D0817322D30
:101A62000813F01D362D8817080088130800F300AC
:101A720083120313081173080A128A151E250A120B
:101A82008A158312031388151A30F200F830F10018
:101A9200F10B492DF20B492D00008312031388111B
:101AA2000800F401F501701C5C2D7208F40703189C
:101AB200F50A7308F50701300310F20DF30DFF3E2E
:101AC200031D5D2D01300310F10CF00CFF3E031DD0
:101AD200642D70087104031D542D7508F1007408FB
:101AE200F00008000A128A15D6240A128A158316F3
:101AF200031391150A128A15D6240A128A15831223
:101B020003131308F200F3017208F4007308F500DE
:101B12000A128A15D6240A128A1570087104031D46
:101B2200962D831603139116992D83160313911282
:101B320011167508F1007408F0000800F701F801A9
:101B420077087507840078080318780A76078312E5
:101B52000313FF000A128A1103200A128A15003A9F
:101B62000319080077087507840078080318780AB3
:101B72007607FF000A128A1103200A128A150A1236
:101B82008A1533260A128A150130F7070318F80A54
:101B92000030F807A12D700871040319F92DF50121
:101BA200F50AF11BE02D01300310F00DF10DFF3E9F
:101BB200031DD52D0130F4007408F507D22D7108EC
:101BC2007302031DE62D70087202031CEE2D7008CD
:101BD200F2027108031CF303F30201300310F10C4B
:101BE200F00CFF3E031DEF2D0130F502031DE02D29
:101BF2007308F1007208F00008000A128A15DF2447
:101C02000A128A15F401F40A01300A128A156B27A6
:101C12000A128A150130F5008030F6000A128A1580
:101C22009F250A128A15F401F40A02300A128A1553
:101C32006B270A128A152230F5008030F6000A124C
:101C42008A159F250A128A153330FD00BB30FC002D
:101C5200DF30FB00FB0B2B2EFC0B2B2EFD0B2B2E58
:101C6200322E0800F40074080F39F1007108F200F6
:101C72007408F039F1007108F30083120313081598
:101C82007308F10004300310F10CFF3E031D442ED3
:101C920071080A128A151E250A128A158312031365
:101CA20088154230F100F10B542E00008312031309
:101CB200881172080A128A151E250A128A158312C1
:101CC200031388154230F100F10B652E00008312D8
:101CD200031388110800F501F60170087104031955
:101CE200A32EF701F70AF11B822E01300310F00D2B
:101CF200F10DFF3E031D772E0130F4007408F70743
:101D0200742E01300310F50DF60DFF3E031D832ED8
:101D120071087302031D8F2E70087202031C982E25
:101D22007008F2027108031CF303F3027514013008
:101D32000310F10CF00CFF3E031D992E0130F70247
:101D4200031D822E7608F1007508F00008000030AD
:101D5200FC000030FB000030FA000030F900701C7B
:101D6200C62E7408F907750803110318013E031DF6
:101D7200FA07760803110318013E031DFB077708D3
:101D820003110318013E031DFC070130F800031084
:101D9200F40DF50DF60DF70DF80BC82E01300310FA
:101DA200F30CF20CF10CF00CFF3E031DD02E730865
:101DB200720471047004031DB02E7C08F3007B08CA
:101DC200F2007A08F1007908F00008000A128A1578
:101DD200DF240A128A15F401F40A01300A128A1564
:101DE2006B270A128A153230F5008030F6000A128B
:101DF2008A159F250A128A15DF300A128A153326A0
:101E02000A128A1543300A128A1533260A128A15D3
:101E1200F401F40A02300A128A156B270A128A1593
:101E22001230F5008030F6000A128A159F250A1238
:101E32008A153330FD00BB30FC00DF30FB00FB0BAA
:101E4200202FFC0B202FFD0B202F272F0800F50140
:101E5200F60171087602031D302F7008750203180F
:101E62000800F701F8018312031388140330F3000A
:101E72006E30F200F20B3B2FF30B3B2F8312031356
:101E82008810D030F200F20B442F0130F70703180C
:101E9200F80A0030F8077808803AFF0080307F02A5
:101EA200031D552FFA307702031C342F0D30F40036
:101EB200AF30F300B630F200F20B5D2FF30B5D2F63
:101EC200F40B5D2F00000130F5070318F60A00300D
:101ED200F6072A2FF7007703031D902F74087F3E21
:101EE200F5007508FA007A08F50004300310F50CC5
:101EF200FF3E031D772F7508F6007608F8007A0872
:101F02000F39F5007508F90078080A128A15382584
:101F12000A128A1579080A128A1538250800023031
:101F22007706031D08007408BF3EF5007508FA0025
:101F32007A08F50004300310F50CFF3E031D9C2FB8
:101F42007508F6007608F8007A080F39F50075086A
:101F5200F90078080A128A1538250A128A157908B2
:101F62000A128A1538250800F601F31FBF2FF2095D
:101F7200F309F20A0319F30AF601F60AF11FC62F52
:101F8200F009F109F00A0319F10A70087104031942
:101F9200F32FF501F50AF11BDA2F01300310F00DD2
:101FA200F10DFF3E031DCF2F0130F4007408F50739
:101FB200CC2F71087302031DE02F70087202031CFC
:101FC200E82F7008F2027108031CF303F3020130D8
:101FD2000310F10CF00CFF3E031DE92F0130F50256
:101FE200031DDA2F76080319FB2FF209F309F20A0F
:0E1FF2000319F30A7308F1007208F0000800EA
:02400E00723FFF
:00000001FF
